:1000000008308A00002800000A108A100A118207AE
:10001000413454342B3443344D3447344C343D3420
:1000200030340D3400340A108A100A11820741342A
:1000300054342B34433443344C344B343F340D3438
:1000400000340A108A100A118207413454342B34C8
:1000500043344D34473444343D3431340D3400346A
:100060000A108A100A1182074A34413443344B344F
:100070005B344234413452346D346B3400340A10F2
:100080008A100A1182075B344534523452344F349B
:1000900052345B3464345B345B3400340A108A10AD
:1000A0000A1182075B344F34563445345234463497
:1000B0004C344F3457345B3400340A108A100A1120
:1000C00082075B344534523452344F3452345B34FB
:1000D00065345B345B3400340A108A100A118207DD
:1000E0005B344F34503441344B3455344A345434F7
:1000F00045345B3400340A108A100A1182075B34DD
:100100005B3456344F344C34423455345B345B34B6
:100110005B3400340A108A100A1182075B345B34A6
:10012000503445344134433445345B345B345B34C0
:1001300000340A108A100A1182075B345B345B3486
:100140004D344F34523445345B345B345B340034CB
:100150000A108A100A1182075B345B345A34453422
:100160005B344A344F345B345B345B3400340A1004
:100170008A100A1182075B3452344F345A344234A5
:100180004934543459345B345B3400340A108A10D7
:100190000A1182075B345B344234553444344934A9
:1001A0004B345B345B345B3400340A108A100A1120
:1001B00082075B345A34413450344F344A34493422
:1001C00054345B345B3400340A108A100A118207FD
:1001D0005B345A3441345334553456344B345534EB
:1001E0005B345B3400340A108A100A11FA3E03189B
:1001F0008A0A82005B345B344D34413452345434C7
:1002000049344E345B345B3400340A148A100A11CA
:1002100082075B345B345334563445344A344434B7
:1002200041345B345B3400340A148A100A118207AB
:100230005B345B3454344F344D34413453345B3489
:100240005B345B3400340A148A100A1182075B3471
:100250005B345B344B34413450344C345B345B346A
:100260005B3400340A148A100A1182075B345B3451
:100270004A3441344B34553442345B345B345B3460
:1002800000340A148A100A1182075B345B344B3441
:1002900041344B344F344E3441345B345B3400349E
:1002A0000A148A100A1182074F34443450344F34F0
:1002B0005634453444345B344E34413400340A14EB
:1002C0008A100A1182075B345B345634413453344C
:1002D00049345B345B345B345B3400340A148A1079
:1002E0000A1182075B345B344F34543441345A343E
:1002F0004B3455345B345B3400340A148A100A11D1
:1003000082075B345B345B345B344A3445345B34A2
:100310005B345B345B3400340A148A100A118207A0
:100320005B345B345B345B34653463345B345B3443
:100330005B345B3400340A148A100A1182075B3480
:100340005B344E34453455344D34493453345B3486
:100350005B3400340A148A100A1182075B345B3460
:100360005B3450345334413454345B345B345B3449
:1003700000340A148A100A1182075B345B34543447
:100380005234553442344B344F345B345B34003494
:100390005230840000080319DD290530F800BF3011
:1003A000F7006400F70BD129F80BCF29F930F700DB
:1003B000F70BD8296400800BCD29003420132008C6
:1003C00083168700831207130830F800000000002E
:1003D0000000F817FA29F813D30C03180717031CA9
:1003E00007137817FA297813F80BEC29000000009E
:1003F0000000071749308400840BFC29000000002E
:100400000000F81BEB29781BF32900340830F700B3
:10041000831686168312861E0F2A83160A2AD70190
:10042000F717202AF713202A0310861A0314D70C73
:100430007717202A7713F70B142A5708F8002D2A6C
:100440004930F71B1430F800F80B242A0000000094
:10045000F71B122A771B1A2A142A0034D1015108DB
:10046000042000380319382AD10AD300DE212F2AAC
:10047000062278080A3C031D382A06227808A600BE
:1004800006227808A700062278080A3C031D432AA2
:1004900026084F3C031D542A27084B3C031D542AB1
:1004A0000130F800572A572A0030F800572A8A15D9
:1004B0000A12A128D1015108353C031C622A0622E8
:1004C000D10A5B2A06227808A60006227808A7002F
:1004D00006227808A80006227808A90006227808D3
:1004E000AA0006227808AB0006227808AC00062293
:1004F0007808AD00A608031D7F2A3030A7003030F1
:10050000A602A7022608093C0318882A0730A6027B
:100510002708093C03188E2A0730A702A60EF030E0
:10052000A6052708A604A808031D982A3030A900AC
:100530003030A802A9022808093C0318A12A073074
:10054000A8022908093C0318A72A0730A902A80E07
:10055000F030A8052908A804AA08031DB12A3030E4
:10056000AB003030AA02AB022A08093C0318BA2AB1
:100570000730AA022B08093C0318C02A0730AB0237
:10058000AA0EF030AA052B08AA04AC08031DCA2A3B
:100590003030AD003030AC02AD022C08093C0318FD
:1005A000D32A0730AC022D08093C0318D92A07309A
:1005B000AD02AC0EF030AC052D08AC042808A70045
:1005C0002A08A8002C08A900AC012C08AB00AA003E
:1005D000D301D1015108033C031C412B0310D60C5D
:1005E000D61726305107840000085605D40026305F
:1005F0005107D7002630510784000008F700530840
:10060000F8000319072B0310F70DF80B032B5708FD
:10061000840077088000D2015308083C5202031876
:10062000162B0310D50CD513D20A0C2B26305107EC
:10063000D70026305107840000085504D900570818
:1006400084005908800026305107D7002630510712
:10065000840000087F39D9005708840059088000B9
:100660005408D500D30A5308083C031D3F2BD3017F
:1006700001305107263E840055088000D601D10A7A
:10068000EA2A26305107840080018A150A12B1280F
:1006900083160611831206110830F80000000000CE
:1006A0000000F817622BF813D20C03180615031C70
:1006B00006117817622B7813F80B542B00000000FA
:1006C000000006150930F7008401840B652BF70B39
:1006D000642BF0308400840B6B2B00000000F81BAF
:1006E000532B781B5B2B0034D1015108212000389B
:1006F00003197E2BD10AD300DE21752B0034D201E1
:100700005208132000380319892BD20AD300DE21A6
:10071000802B06227808223C031D892BD101510829
:100720000B3C031C962B0622D10A8F2B062278083D
:10073000A60006227808A700A8018A150A12FA2C3A
:1007400083164708C9004608CA004808003C031839
:10075000B52B4A08840049080002031DB22B4A0841
:10076000F800B72BCA0AC803A52B0030F800831283
:10077000003410308316CA00F701FA01C70CC60C0A
:10078000031CC82B4808F7070318FA0A4908FA0798
:10079000FA0CF70CF90CF80CCA0BBE2B83128A1159
:1007A0000A120B2DD701D80130308316A00031304A
:1007B000A1003230A2003330A3003430A400353021
:1007C000A5003630A6003730A7003830A8003930F1
:1007D000A9006130AA006230AB006330AC00643025
:1007E000AD006530AE006630AF006730B0006830F5
:1007F000B1006930B2006A30B3006B30B4006C30C5
:10080000B5006D30B6006E30B7006F30B800703094
:10081000B9007130BA007330BB007430BC00753061
:10082000BD007630BE007730BF007830C000793030
:10083000C1007A30C200C30183125108D4005408A9
:1008400084000008203C031D272CD40A1F2C5408C8
:10085000840000082D3C0319332C54088400000840
:100860002B3C031D382C5408D40A84000008392C72
:100870002B30D90059082D3C031D492CD2080319EF
:10088000452C52088400510880000030F800F9001F
:10089000552DD31B542C530B4E2C542CD31B602C96
:1008A0005308243C0318602CD20803195B2C52080F
:1008B0008400510880000030F800F900552DC62C46
:1008C000D30803199D2C5308103C031D7D2C54089C
:1008D00084000008303C031D7D2C01305407840047
:1008E0000008783C03197B2C013054078400000871
:1008F000583C031D7D2C0230D4075308083C031DCF
:10090000892C540884000008303C031D892C0130D8
:10091000D4075308023C031D9C2C54088400000893
:10092000303C031D9C2C0130540784000008623CBD
:10093000031D9C2C0230D407C62C540884000008E8
:10094000303C0319A62C0A30D300C62C01305407C2
:1009500084000008783C0319B42C0130540784004B
:100960000008583C031DB92C1030D3000230D407C6
:10097000C62C0130540784000008623C031DC42CBF
:100980000230D300D407C62C0830D3005408D50059
:10099000540884000008303C031DD02CD40AC82C15
:1009A000540884000008DA00403C0318DE2C5A0882
:1009B0005A3C031CDE2C5A082038DF2C5A08DB0076
:1009C000A0308316C60083125A088316C70083120C
:1009D00053088316C8008312A0237808D600D608CF
:1009E00003193B2DFA015308F700D31BFA03DA0071
:1009F0007A08DB0058088316C7008312570883164D
:100A0000C60083127A088316C90083125A08831617
:100A1000C8008312B92B7808DB00A0305602FA0117
:100A20007807F8000318FA0A7908FA077808D70057
:100A30007A08D800D40A540884000008DA00403C40
:100A40000318292D5A085A3C031C292D5A0820380E
:100A50002A2D5A08DB00A0308316C60083125A08DC
:100A60008316C700831253088316C8008312A0237D
:100A70007808D600EF2C54085502031D4A2DD208E1
:100A80000319462D52088400510880000030F800F8
:100A9000F900552DD2080319512D5208840054082D
:100AA00080005708F8005808F9008A150A12032D2B
:1010000084011F3083052013200883168700831274
:101010000717831606118312061583161F149F14D3
:101020001F159F1107309C00FF308312A000A10103
:101030000130A200A301A401A50183161F149F146F
:101040001F159F1183121F109412A01220088316DF
:101050008700831220162008831687008312A011B0
:101060002008831687000130831294000030831615
:1010700094000108C73908388100831290010030BC
:10108000F80005389200FF30831692008312201179
:10109000200883168700831207110C309700A010D8
:1010A000200883168700831287100C309D000730BC
:1010B00083169C00050864000E30F700F70B5E28CD
:1010C000000000001C0883120D1383169D010F30D1
:1010D000F700073083128101813084000008F03965
:1010E0000738800064000008F739F719F0397704F1
:1010F000800095019B01831605128312051296301C
:10110000D2008A11C8218A1583160512831205168A
:101110009630D2008A11C8218A15831605128312CF
:1011200005129630D2008A11C8218A15831605123D
:10113000831205169630D2008A11C8218A158A11A9
:101140002E2A8A15F8080319AF280430D100FA3086
:10115000D2008A11C8218A15D10BA728F82C8A1130
:101160005A2A8A152608603C0318BD2826087A3CAE
:10117000031CBD282608DF39BE282608413C031D74
:101180000129643095009B002830D100FA30D2004C
:101190008A11C8218A15D10BC628D10151088A119C
:1011A00030208A1500380319DB28D10AD2008A11B1
:1011B00048238A15CE280830D100FA30D2008A118F
:1011C000C8218A15D10BDD28D10151088A113020A0
:1011D0008A1500380319F228D10AD2008A1148234F
:1011E0008A15E5281430D100FA30D2008A11C821BE
:1011F0008A15D10BF42895019B018A1174238A1555
:10120000322D2608603C03180C2926087A3C031C62
:101210000C292608DF390D292608423C031D6029C8
:10122000643095009B002830D100FA30D2008A113A
:10123000C8218A15D10B1529CE014E08013C031C8B
:101240005129D10151088A113F208A15003803190C
:101250002F29D10AD2008A1148238A152229083061
:10126000D100FA30D2008A11C8218A15D10B312958
:10127000D10151088A114E208A15003803194629D8
:10128000D10AD2008A1148238A1539290830D100A1
:10129000FA30D2008A11C8218A15D10B4829CE0A0A
:1012A0001D291430D100FA30D2008A11C8218A15C4
:1012B000D10B532995019B018A1174238A15322D74
:1012C0002608603C03186B2926087A3C031C6B290E
:1012D0002608DF396C292608433C031DD6296430D3
:1012E00095009B002830D100FA30D2008A11C82125
:1012F0008A15D10B7429CE014E08013C031CC72965
:10130000D10151088A115D208A15003803198E29F0
:10131000D10AD2008A1148238A1581290830D100C8
:10132000FA30D2008A11C8218A15D10B9029D10137
:1013300051088A116C208A1500380319A529D10A91
:10134000D2008A1148238A1598290830D100FA3032
:10135000D2008A11C8218A15D10BA729D1015108C1
:101360008A117B208A1500380319BC29D10AD200C2
:101370008A1148238A15AF290830D100FA30D200EB
:101380008A11C8218A15D10BBE29CE0A7C290C30BE
:10139000D100FA30D2008A11C8218A15D10BC9298F
:1013A00095019B018A1174238A15322D2608603C11
:1013B0000318E12926087A3C031CE1292608DF39B5
:1013C000E2292608443C031D252A643095009B0031
:1013D0002830D100FA30D2008A11C8218A15D10BE9
:1013E000EA29D10151088A118A208A150038031987
:1013F000FF29D10AD2008A1148238A15F229083020
:10140000D100FA30D2008A11C8218A15D10B012AE5
:10141000D10151088A118A208A1500380319162A29
:10142000D10AD2008A1148238A15092A0C30D1002A
:10143000FA30D2008A11C8218A15D10B182A9501D9
:101440009B018A1174238A15322D2608603C0318EB
:10145000302A26087A3C031C302A2608DF39312A34
:101460002608453C031D842A643095009B002830E3
:10147000D100FA30D2008A11C8218A15D10B392A3D
:10148000CE014E08013C031C752AD10151088A1176
:1014900099208A1500380319532AD10AD2008A11DB
:1014A00048238A15462A0830D100FA30D2008A1122
:1014B000C8218A15D10B552AD10151088A11A820BB
:1014C0008A15003803196A2AD10AD2008A114823E2
:1014D0008A155D2A0830D100FA30D2008A11C8215D
:1014E0008A15D10B6C2ACE0A412A1430D100FA3069
:1014F000D2008A11C8218A15D10B772A95019B0148
:101500008A1174238A15322D2608603C03188F2A0D
:1015100026087A3C031C8F2A2608DF39902A2608E1
:10152000463C031DE32A643095009B002830D1001F
:10153000FA30D2008A11C8218A15D10B982ACE011F
:101540004E08013C031CD42AD10151088A11B7204E
:101550008A1500380319B22AD10AD2008A11482309
:101560008A15A52A0830D100FA30D2008A11C82184
:101570008A15D10BB42AD10151088A11C6208A15C7
:1015800000380319C92AD10AD2008A1148238A15C2
:10159000BC2A0830D100FA30D2008A11C8218A153D
:1015A000D10BCB2ACE0AA02A1430D100FA30D200B7
:1015B0008A11C8218A15D10BD62A95019B018A115F
:1015C00074238A15322D2608603C0318EE2A26085B
:1015D0007A3C031CEE2A2608DF39EF2A2608473C0E
:1015E000031D422B643095009B002830D100FA3057
:1015F000D2008A11C8218A15D10BF72ACE014E08D4
:10160000013C031C332BD10151088A11D5208A15C6
:1016100000380319112BD10AD2008A1148238A15E8
:10162000042B0830D100FA30D2008A11C8218A1563
:10163000D10B132BD10151088A11E4208A150038EF
:101640000319282BD10AD2008A1148238A151B2B93
:101650000830D100FA30D2008A11C8218A15D10B86
:101660002A2BCE0AFF2A1430D100FA30D2008A1178
:10167000C8218A15D10B352B95019B018A11742342
:101680008A15322D2608603C03184D2B26087A3C1B
:10169000031C4D2B2608DF394E2B2608483C031D22
:1016A000FD2B643095009B002830D100FA30D20029
:1016B0008A11C8218A15D10B562BCE014E08013C48
:1016C000031CEE2BD10151088A11F3208A15003832
:1016D0000319702BD10AD2008A1148238A15632B73
:1016E0000830D100FA30D2008A11C8218A15D10BF6
:1016F000722BD10151088A1105218A15003803196E
:10170000872BD10AD2008A1148238A157A2B0830F8
:10171000D100FA30D2008A11C8218A15D10B892B49
:10172000D10151088A1114218A15003803199E2B02
:10173000D10AD2008A1148238A15912B0830D10092
:10174000FA30D2008A11C8218A15D10BA02BD10101
:1017500051088A1123218A1500380319B52BD10AA3
:10176000D2008A1148238A15A82B0830D100FA30FC
:10177000D2008A11C8218A15D10BB72BD10151088B
:101780008A1132218A1500380319CC2BD10AD200D4
:101790008A1148238A15BF2B0830D100FA30D200B5
:1017A0008A11C8218A15D10BCE2BD10151088A117B
:1017B00041218A1500380319E32BD10AD2008A117E
:1017C00048238A15D62B0830D100FA30D2008A116E
:1017D000C8218A15D10BE52BCE0A5E2B0C30D10027
:1017E000FA30D2008A11C8218A15D10BF02B95014D
:1017F0009B018A1174238A15322D2608603C031838
:10180000082C26087A3C031C082C2608DF39092CF2
:101810002608493C031DA22C643095009B0028300B
:10182000D100FA30D2008A11C8218A15D10B112CAF
:10183000CE014E08013C031C922CD10151088A11A3
:1018400050218A15003803192B2CD10AD2008A1195
:1018500048238A151E2C0830D100FA30D2008A1194
:10186000C8218A15D10B2D2CD10151088A115F2175
:101870008A1500380319422CD10AD2008A11482354
:101880008A15352C0830D100FA30D2008A11C821CF
:101890008A15D10B442CD10151088A116E218A1569
:1018A00000380319592CD10AD2008A1148238A150D
:1018B0004C2C0830D100FA30D2008A11C8218A1588
:1018C000D10B5B2CD10151088A117D218A1500387A
:1018D0000319702CD10AD2008A1148238A15632C6F
:1018E0000830D100FA30D2008A11C8218A15D10BF4
:1018F000722CD10151088A118C218A1500380319E4
:10190000872CD10AD2008A1148238A157A2C0830F4
:10191000D100FA30D2008A11C8218A15D10B892C46
:10192000CE0A192C0C30D100FA30D2008A11C8210D
:101930008A15D10B942C95019B018A1174238A1569
:10194000322DF82C643095009B002830D100FA30FD
:10195000D2008A11C8218A15D10BA72CD1015108B8
:101960008A119B218A1500380319BC2CD10AD20098
:101970008A1148238A15AF2C0830D100FA30D200E2
:101980008A11C8218A15D10BBE2CD10151088A11A8
:10199000AA218A1500380319D32CD10AD2008A1142
:1019A00048238A15C62C0830D100FA30D2008A119B
:1019B000C8218A15D10BD52CD10151088A11B92122
:1019C0008A1500380319EA2CD10AD2008A1148235B
:1019D0008A15DD2C0C30D100FA30D2008A11C821D2
:1019E0008A15D10BEC2C95019B018A1174238A1561
:1019F0008A117F2B8A152630D1004F30D2000A3051
:101A0000D3008A11D22B8A157808D00050081D3CCB
:101A100003180E2D5008203C0318222D5008023CBC
:101A20000318222D50082C3C03181A2D50082F3C67
:101A30000318222D50080E3C0318262D5008113C87
:101A4000031C262D643095009B00282D95019B01D9
:101A50000430D100FA30D2008A11C8218A15D10B86
:061A60002A2D7B28630023
:02400E003E3F33
:00000001FF
